:03000000020C00EF
:03000300021A03DB
:03000B00021A06D0
:03001300021A09C5
:03001B00021A0CBA
:03002300021A0FAF
:03002B00021A12A4
:03003300021A1599
:03003B00021A188E
:03004300021A1B83
:03004B00021A1E78
:03005300021A216D
:03005B00021A2462
:03006300021A2757
:03006B00021A2A4C
:03007300021A2D41
:03007B00021A3036
:03008300021A332B
:03008B00021A3620
:03009300021A3915
:03009B00021A3C0A
:0300A300021A3FFF
:100C0000787FE4F6D8FD9000007F007E20E4F0A31A
:0A0C1000DFFCDEFA75814A020C5584
:102C1D0002000205020B02100216021C02220228FB
:102C2D00022E0234023A02400247024D0253025A6A
:102C3D0002600267026E0274027B028202890290B8
:102C4D000297029F02A602AD02B502BC02C402CCDD
:102C5D0002D402DB02E302EB02F402FC0304030DD7
:102C6D000315031E0326032F03380341034A0353A1
:102C7D00035D0366036F03790383038C039603A03F
:102C8D0003AB03B503BF03CA03D403DF03EA03F4A5
:102C9D00FFFF064003200190010A00C80085006473
:0A2CAD000050003500280020001A36
:10202E004105AF054304200105B04304230105B06B
:10203E004106B100C1074106B0004204AD000041A7
:10204E00042600C1034104940041041C00410457BE
:10205E0000C104C102C101C10BC105C106C10941C4
:10206E00042F00C10CC100410491004104520041F3
:10207E00041B004204A9000042049900004204928D
:10208E0000004404A000000000410455F0420495F5
:10209E000000C1084404A50000000041049800415E
:1020AE00045900410458004204530000410434AA6C
:1020BE004104A4AA41044F00420450000041049B75
:1020CE00FF41048FFF410435FF41045600440430A4
:1020DE000800000044049C04F1BBCD44042700001A
:1020EE0000004404140000000044042B0000000013
:1020FE0044040E000000004204AB2EE04204120025
:10210E0000C18A43045A3132304104900044040A1B
:04211E00000014CBDE
:101D7D0074362FF582E43404F5832290086AE02549
:101D8D00E0242EF582E43407F583E0FEA3E0FF9016
:101D9D00086BE025E0245DF582E43404F583EEF074
:101DAD00A3EFF090086BE004F022EF25E0241FF57F
:101DBD0082E43407F583229007EE1210709007EE3F
:101DCD000210239007C3E0FF900843E06F229008B4
:101DDD006AE0FFC3941922EF25E0242EF582E43446
:101DED00072290086AE004F02290041D7B017A041A
:101DFD0079AF021100E025E0249DF582E4342CF545
:101E0D0083E493FE74019322FFE43EFEE43DFDE482
:101E1D003CFC0210707FFF7EFF7D0F7C009004A0C4
:101E2D0002102FE4FCFDFE12102F020EB8EF25E07C
:101E3D00245DF582E43404229007EA1210709007B5
:101E4D00EA02102374602FF582E43407F58322E053
:101E5D002FFFC364809480229004A0021023E475A8
:101E6D00F001020E71900844E0FFA3E0FDA3E0FB3A
:101E7D002212102FC3020FEB90086BF0A3F0900805
:101E8D006AF02290041D0210C97C007D0CAE020286
:101E9D000E1CE0FEA3E0FFE422ED543FF0EDAE0496
:101EAD007806223395E08DF0120E71D3227B017AE4
:101EBD000579B0021100E475F0011210E9740122E8
:0D1ECD0090071DE064012290041402102310
:10382600121E90C003C002C0019004181210C9D025
:1038360082D083D0E06B7008E965827003EA658305
:0838460060037F01227F0022D4
:1038C300121E90120DB2FF90041E121E6B121E9058
:1038D30074019005AF6B7008E965827003EA658334
:0538E3007003121DF648
:0138E80022BD
:053E6B00C205D2062291
:10344F0090071DE0FF900459F0B4010A90071D7416
:10345F0002F0C20C8014EFB4020890071D7401F043
:10346F008008EF700590071D04F0900459E0B40137
:10347F000A90071DE0B40203123E6B200609900765
:0D348F001DE0B40202E4F0121A1B0217BF88
:0833B00090071CE06401703677
:1033B80090072CE0FAA3E0FBFF121E96900889EF15
:1033C800F0AF03121E96AF05A3EFF0C39406900862
:1033D80089E05002800204F075F00CA4FF90072CDD
:0633E800E5F0F0A3EFF098
:1033EE0090071CE004F0D394024002E4F0121A1B82
:0333FE000217BFF4
:103A8800200809A203B39203D208800CC203C20320
:0B3A9800123DF8E4900498F00217BF04
:1030E000900498E06023900426E0FF700404F080D0
:1030F00038EFB401089004267402F0802CEF6402CB
:10310000702790042604F08020900426E0FF7004CD
:1031100004F08015EFB40107E4900426F0800AEF74
:10312000B402069004267401F0900426E07005C2F3
:0F31300003123DF890071DE0700204F00217BF74
:10378000D390072DE0940090072CE094004018900F
:10379000071CE090072CB4020774FF75F0F4800456
:0A37A00074FFF5F0120E71021A1BFF
:1037D400C390072DE0945490072CE0940050179068
:1037E400071CE090072CB40206E475F00C8004E496
:0937F40075F001120E71021A1B9E
:1022AB009007DB121E9FFCFD9007F2121070900737
:1022BB002A121E9F2FFFEE34F8FEE434FFFDE434A8
:1022CB00FFFC9007F2121E349007F6121070900765
:1022DB00F6121023E4FB7A08F9F812352F9007F663
:1022EB0012107090072DE02418FF90072CE034009B
:1022FB00FE7C007DC3120E0A30090874482FFF7450
:10230B00123EFEEF7802CEC313CE13D8F9FFE4FCD6
:10231B00FD121E459007F612102F120E9D121E4530
:10232B00EC33500A9007EA12107C00000000E47FA7
:10233B00917E14FDFC9007EA12102FD3120FD5409B
:10234B000A9007EA12107C00001491121E4B121D0A
:10235B00C4E47B207A01F9F8120EB8121DC4E47B99
:10236B00917A14F9F8120F43121DC4EF241A900737
:10237B00EE121E15E47B40FAF9F8121DCA120F4338
:10238B00AB07121DCAEF543FFFC374049BFEEF252E
:10239B00E0241DF582E4342CF583E493FD74019362
:1023AB009004ADCDF0A3EDF0AF069004ADE0FEA32D
:1023BB00E0A807088005CEC313CE13D8F9F0EE9032
:0323CB0004ADF06E
:0123CE0022EC
:0A3DF8007F19900436E4F0A3DFFC0D
:013E0200229D
:031A1500023DF897
:103CA700E4D39F500DEFC394045007EF2498FF12FD
:033CB70034E722CD
:0435B000AD07AC06B1
:1035B400ED4C70079005AFE02407F090088C121EC4
:1035C400A6CEA2E713CE13D8F8FDAC06543F90085C
:1035D4008BF07F971234E790088CE0FF1234E79069
:0735E400088BE0FF0234E751
:103CCD0090089FEFF07F941234E790089FE0FF0279
:023CDD0034E7CA
:1039F900900727E004F0C394044002E4F0900727FD
:0D3A0900E0FF123CA77FE91234E7021A1B10
:10399900900727E0600414F080069007277403F06D
:1039A900900727E0FF123CA77FE91234E7021A1BB0
:103ABE009008A0EFF0BF1A05123A88800A9008A06D
:0A3ACE00E0B419031230E00217BF44
:102DE4009008A1EFF064196004E0B41A089008A1F7
:102DF400E0FF023ABE3003359008A1E0FFD39418F7
:102E040050047E0180027E00E4D39F50047F018041
:102E1400027F00EF5E600B9008A1E02436121D8053
:102E2400E4F0123D8AEF704CC2030217BF900426EF
:102E3400E06402603F9008A1E0FFD3941850047E40
:102E44000180027E00E4D39F50047F0180027F0052
:102E5400EF5E60209008A1E0FF64116017EF641238
:102E64006012121E51E0600C9008A1E02436121D7D
:052E7400807401F02252
:10384E00900426E07020EFD3941850047E0180027D
:10385E007E00E4D39F50047D0180027D00ED5E600A
:07386E0005121D7DE4F022AC
:0D3DD200900497E0C394185003E004F02221
:093E3A00900497E0600214F022EC
:103B8B00E4D39F5012EFC39419500C121E51EDF059
:083B9B007005121D7DE4F0220B
:0535EB00900880EFF0E4
:1035F000900882121EA6CEC313CE13D8F9FDAC06D6
:10360000543F900881F07F901234E7900880E0FFEB
:103610001234E7900882E0FF1234E7900881E0FF5F
:033620000234E78A
:103A160090088DEFF0A3EDF07F951234E790088DB6
:0D3A2600E0FF1234E790088EE0FF0234E765
:103D5A00121DE4F583ECF0A3EDF01235EB021A1B09
:103CDF009008A2EFF07F8C1234E79008A2E0FF0269
:023CEF0034E7B8
:103CF1009008A3EFF07F8D1234E79008A3E0FF0254
:023D010034E7A5
:052E7900E4900875F073
:102E7E00900875E0FF121DE5F583E0FCA3E0FD90E0
:102E8E000876ECF0A3EDF01235EB900875E0FF2418
:092E9E0060121E54E0FD123A1608
:102EA700900875E004F0E0C3941940CBE4900874EF
:102EB700F0900874E0FFC39404501A123CA79008DE
:102EC70074E0121DB8E0FEA3E0FF1235B09008745D
:102ED700E004F080DC900727E0FF900874F0123CD4
:102EE700A790071EE0FF123CCD900728E0FF123C99
:0E2EF700DF900729E0FF123CF17FE91234E77B
:012F050022A9
:0C3DEC00EF6003D38001C392010217BFF7
:103C7F007406D39F5009EF94075004D20B8002C2F1
:043C8F000B0217BF4E
:0A335C00E4D39F504EEF941950493E
:10336600121DE4F583E0FBA3E090088FCBF0A3EBFE
:10337600F0ED90088F121EB0900890E094C6900869
:103386008FE06480948340077403F0A374C6F0C38F
:1033960090088FE0648094805004E4F0A3F09008D5
:0933A6008FE0FCA3E0FD123D5A8A
:0133AF0022FB
:0B3E030090071EEFF0123CCD021A1BCE
:103AD80090071E121E5C5002E4FFD3EF64809484AA
:0A3AE80040027F04123E03021A1B85
:0B3E0E00900728EFF0123CDF021A1BA7
:0B3E1900900729EFF0123CF1021A1B89
:103AF200900728121E5C5002E4FFD3EF6480948C7E
:0A3B020040027F0C123E0E021A1B57
:103B0C00900729121E5C5002E4FFD3EF6480948C62
:0A3B1C0040027F0C123E19021A1B32
:10112F009007C3745BF075FFDE75FFAD123B7290D5
:10113F0007AF12107C007C9D0A9007B312107C0041
:10114F00000FA09007B712107C000007F99007BBA3
:10115F0012107C0000F807121A15123727123A5096
:10116F00123A33123935123D38123D03123D6A12CD
:10117F003E4B123D15121A219007BF12107C05D756
:10118F005C80D2AF43A82043A81075E60875E70628
:10119F001217BFD2857E017F009005B074AAF0A30D
:1011AF00DFFCDEFA7E017F00121DF690041812118B
:1011BF0000123573E490071AF0123BBB123875EF2B
:1011CF00606612349CEF12110911FA0111FF02121D
:1011DF001003121504121A05120406121F07122902
:1011EF0008122409122E0A0000123112344F8032D5
:1011FF001233B0802D9007C3E0FF7D031239B98001
:10120F00211239F9801C123A8880171230E08012AF
:10121F00123978800D12378080081237D48003126C
:10122F003E59123875EF709A123826EF6401600339
:03123F000213B2E5
:101242001238C39007C4EFF020E703021304E090C2
:101252000455F0121109129889129C8A12E0A81200
:10126200E4A912E8AA12ECAB12F0AC12F4AD12F837
:10127200AE12FCAF12D8B212D4B312B0B412B4B5DB
:1012820012BCB612C0B712C8B812CCB912A4BA12A4
:10129200AABC000013B27F018002E4FF123DEC02FF
:1012A20013B2123E2F0213B2122E790213B27F0131
:1012B20080027FFF123AD80213B27F0180027FFFC1
:1012C200123AF20213B27F0180027FFF123B0C023C
:1012D20013B27FFF80027F01123AA30213B27F0191
:1012E200801A7F1080167F4080127F7F800E7FFFE2
:1012F200800A7FF080067FC080027F811231F9026E
:1013020013B2900455E0121109133682134083136D
:10131200958B139F8E13A88F134AA01353A1135CAE
:10132200A21365A3136EA41377A51380A61389A72E
:10133200000013B29007C4E0FF122DE48072900700
:10134200C4E0FF12384E80689007C4E0FF7D018040
:101352003D9007C4E0FF7D1080349007C4E0FF7D1C
:1013620040802B9007C4E0FF7D7F80229007C4E07D
:10137200FF7DFF80199007C4E0FF7DF08010900789
:10138200C4E0FF7DC080079007C4E0FF7D81123377
:101392005C801D9007C4E0FF123C7F80139007C45D
:1013A200E0FFE4FD80079007C4E0FF7D01123B8B64
:1013B2001236C7EF70030214B9300122900842E0DE
:1013C200146010047018900843E090071AF0123B62
:1013D200BB800B900843E090071AF0123E2F900852
:1013E20042E0FFB40B02D202EF6431701E121DD034
:1013F200701912390F50FB1214C7A3E09007FDF0C9
:1014020012273712390F50FB1214DB900842E064A6
:10141200327018121DD0701312390F50FB1214C7FC
:1014220012280412390F50FB1214DB900842E064B8
:101432002D702A121DD0702512390F50FB9007C350
:10144200E0FF123C5512390F50FB121E72122CB7DC
:1014520012390F50FB9007C3E0FF123C4090084244
:10146200E0642E702A121DD0702512390F50FB90A5
:1014720007C3E0FF123C5512390F50FB121E7212C5
:101482002D4E12390F50FB9007C3E0FF123C4090E3
:101492000842E030E7097B017A0879411236F79079
:1014A2000842E0B41405D2011217BF900842E0B41A
:1014B2001505C2011217BF2000030211CB122E79AB
:0514C200C2000211CB85
:1014C7009007C3E0FF123C55900844E0FFA3E0FDFE
:0D14D700A3E0FB229007C3E0FF123C40227F
:103D2700121DB7ECF0A3EDF0AE04FF1235B0021A86
:013D37001B70
:1031F900900727E0FEE4D39E5051EEC39404504B50
:10320900EE121DB8E0FDA3E0900891CDF0A3EDF01A
:10321900EFFD900891121EB0900892E094F4900886
:1032290091E06480948140077401F0A374F4F0C3C1
:10323900900891E0648094805004E4F0A3F0AF0614
:0B324900900891E0FCA3E0FD123D277F
:013254002257
:0E3DA800900727EFF0123CA7121A1B0217BF5C
:103AA300900727E02FFFD36480F8748098500BC3EE
:0A3AB300EF648094845003123DA8D4
:013ABD0022E6
:063E5900A209B392092248
:103D6A00E4F58475D84075D98375DA3175DB31226B
:073E4B00E4F58475D10322A8
:10393500AF8475840F75A43475A5FC75A6FF75A7AE
:10394500FF75E11775E340E4F59075A0FFF5B08FBD
:0139550084ED
:01395600224E
:103A5000AF84E4F58475C9E775CBF875CA0785CBE3
:0B3A6000CD85CACC75C804D2AD8F84A0
:013A6B002238
:103A3300AF8475840275C9E775CB6075CA7F85CA83
:0C3A4300CC85CBCD75C80443E7048F840C
:013A4F002254
:103B4000AF84E4F584758920758E10758D40F58BF2
:083B50004388408F8443A880E4
:013B5800224A
:103D3800123B40E4F584759850F584D2AC43A81042
:013D48002258
:103D0300E4F584759A4075F809759D01759D10C297
:023D1300FA2292
:1034E7009006B1E07002740160F6C2AC900420E46B
:1034F70075F0011210D2EF120DF89004201210C9C6
:1035070074019006B06B7008E965827003EA658301
:103517007006900420121EBA9006B1E004F020074E
:0835270004D207D299D2AC22B4
:031A0F0002259914
:10259900C0E0C0F0C083C082C0D075D000C000C008
:1025A90001C002C00375840030982FC298900418A6
:1025B9001210C9E599120DF8900418121EC390055E
:1025C900AF6B7008E965827003EA65837006900451
:1025D90018121DF99006B0E004F030996F9006B119
:0325E900E060654A
:1025EC009004231210C9120DB29008A4F0C29924C1
:1025FC00EC601214601714601C2488701E9005AFD8
:10260C00740BF080169005AF7407F0800E9005AF38
:10261C007405F080069005AF7403F09008A4E0F503
:10262C00999006B1E014F0900423121EC39006B0EA
:10263C006B7008E965827003EA6583700C90042363
:03264C00121EBAA1
:10264F008004C299C207D003D002D001D000D0D0ED
:09265F00D082D083D0F0D0E0322B
:10395700C2069004A012107C00000000E4900492BC
:10396700F0A3F0900426F090071DF0123DF802171F
:01397700BF90
:102F060030053A900728E070028028121E22C3126C
:102F16000FD55029121E2A900728121E02FFE4FC24
:102F2600FD120E9D9004A0121070121E22D3120FD5
:102F3600D5400A9004A012107C000FFFFF30063126
:102F4600121E65EC33402A121E65C006C0079007A4
:102F560029121E02FBAA06E4F9F8D007D006120EC3
:102F6600AA9004A0121070121E65EC335003123999
:102F760057121E65780412100F900492EEF0A3EF1C
:022F8600F02237
:031A12000228CCDB
:1028CC00C0E0C0F0C083C082C0D075D000C000C0D2
:1028DC0001C002C003C004C005C006C007C2CF308F
:1028EC00082CE47FD07E07FDFC9004A5121E7E50C0
:1028FC00119004A5121023EF24019004A5121E15AB
:10290C00800CC2089004A512107C000000009004FA
:10291C0050E0FEA3E0FFEE702BEF14600C14600E81
:10292C0024027020123E52801B1221738016122F2B
:10293C0006900457E0600D90041CE0600414F080D5
:10294C0003123B26900450121E6BFEC3E5F0940359
:10295C00EE648094804007900450E4F0A3F01222BF
:10296C00AB1217BFD007D006D005D004D003D002CD
:0F297C00D001D000D0D0D082D083D0F0D0E032C4
:1038E900200C17D20CD205E4900492F0A3F09004B6
:1038F900A012107C00000000C2067F3290045D74A3
:05390900FFF0A3DFFC4C
:01390E002296
:103C1600121ECD6002C2057F3290045D74FFF0A3D0
:053C2600DFFC023DF887
:103255009008A5EFF090049C121E309004271210E0
:10326500709008A5E0FF900430121E3090040E12F5
:103275001070121ED490042712102F120E9D801A62
:1032850090040E121023900414121E7E4014121E78
:10329500D490040E12102F120EAA9004141210705E
:0B32A50080DE121ED4781B120FFC22EA
:1014E400900498E0900456F0E4900498F090086A10
:1014F400F0121DDB5013121D7DE0600890049874F7
:1015040001F08005121DEF80E8900456E070099008
:101514000498E060031238E9900498E070047F01B5
:1015240080027F00900456E05F6003123C16900432
:1015340098E0700302179390049BE030E727E4904F
:10154400086AF0121DDB501D121D7DE06012900729
:101554001EE06404600F90086AE090049BF080052C
:10156400121DEF80DEE490086AF0121DDB501512A4
:101574001D7DE0600A90086AE090048FF0800512F7
:101584001DEF80E690086A7418F090086AE0601A0B
:101594002436121D80E0600A90086AE0900435F059
:1015A400800890086AE014F080E090071EE064046C
:0215B400703C89
:1015B600121E85121DDB5012121D7DE06007121DE2
:1015C60088A3E004F0121DEF80E990086BE0FFC3EA
:1015D6009419500D121E3AF583E4F0A3121DAF8044
:0C15E600E990086CE0FF1232550216423A
:0815F20090071EE06403705332
:1015FA00121E85121DDB5012121D7DE06007121D9E
:10160A0088A3E004F0121DEF80E990086BE0FFC3A5
:10161A009419500D121E3AF583E4F0A3121DAF80FF
:10162A00E912362390086DEEF0A3EFF090086CE013
:10163A00FD7C00120E1CAF0590049BEFF0121E3BBE
:03164A0002172064
:10164D0090071EE0FF7006900899F0800AEFB40134
:10165D00069008997401F0900899E0FF7036900893
:10166D006AF090049BE004F0E0B41902E4F09008F5
:10167D006AE0C39419505D90049BE02436121D80DE
:10168D00E07051121DEF90049BE004F0E0B419DE00
:10169D00E4F080DAEF6401703B90086AF090049BEF
:1016AD00E0600414F0800590049B802390086AE0AC
:1016BD00C39419501F90049BE0FF2436121D80E047
:1016CD007012121DEFEF90049B600414F080DD7416
:1016DD0018F080D890071EE064027030900899E0F1
:1016ED00FF7014900435E0FE90049BE0B506089061
:1016FD0008997401F08015EFB4011190048FE0FF8B
:10170D0090049BE0B50705E4900899F090049BE0E8
:10171D00121DE5F583E0FFA3E0900499CFF0A3EF50
:10172D00F0900727E0FF90086AF0900499E0FCA381
:10173D00E0FD121DB7E0FEA3E02DFDEE3CFC7406AE
:10174D002DFD74FF3CFCC3648094805003E4FCFDCC
:10175D00D3ED94C6EC6480948340047C037DC6AFC6
:10176D0005900499ECF0A3EFF0900499E0FEA3E04E
:10177D007806C333CE33CED8F9F0EE900499F0A3AA
:10178D00E054F0F0800690049B74FFF0E490049117
:10179D00F090041BF0900498E07003300613E49071
:1017AD00042FF090049104F0900452F090041B0467
:0117BD00F03B
:0117BE002208
:031A330002298BFA
:10298B00C0E0C0F0C083C082C0D075D000C000C012
:10299B0001C002C003C004C005C006C007C2CFC33C
:1029AB00900413E094E8900412E094035016121E66
:1029BB006B900412E07004A3E064C87007300A0443
:1029CB00C20AD200121ECD6011900426E0FF6401F2
:1029DB006008EF6402600330063690071CE070302D
:1029EB009004ADE0FEA3E0FFC39004ACE09FFF902A
:1029FB0004ABE09EFEF0A3EFF0D39400EE64809462
:102A0B0080500D1214E49004AB742EF0A374E0F01C
:102A1B00D007D006D005D004D003D002D001D0000F
:0B2A2B00D0D0D082D083D0F0D0E032B9
:10397800121ECD6011900426E0FF64016008EF6418
:1039880002600330060A90071CE0B401031214E435
:01399800220C
:073E5200E4F58443E81022AF
:1021730090042FE004F0C394034002E4F090042F92
:10218300E0FF245AF582E43404F583E0900848F034
:10219300EF14605414700302221B24026003022212
:1021A30068900499121E9FFCFD7B64FAF9F8120EE5
:1021B300B8E47B6AFAF9F8120F4390084B121070D7
:1021C30090040412102390084B121E7E7003022207
:1021D300AA90084B12102390040412107090084B1D
:1021E300121023AC06EF8029900402E0FEA3E0FF67
:1021F300900492E0FCA3E06F7002EC6E7003022285
:10220300AA900492E0FEA3E0FF900402EEF0A3EF95
:10221300F090084AF0EC8049900452E0600414F016
:102223008013900491E0600614F074FF8001E49041
:1022330004A9F0A3F090041BE0600214F09004A939
:10224300E0FEA3E0FF900408E06E7003A3E06F607C
:1022530056900408EEF0A3EFF090084AF09004A91A
:10226300E0900849F0E4F584C2FAFF0FEFB464FB91
:10227300E59A20E7FBE4F59BE59A20E7FB90084805
:10228300E0F59BE59A20E7FB900849E0F59BE59A8A
:1022930020E7FB90084AE0F59BE59A20E7FBE4FF83
:0722A3000FEFB464FBD2FA57
:0122AA002211
:103623007F217EF17D7D7C0090040A121E34EF24FD
:10363300F3FFEE3490FEED3424FDE43CFC90040AE9
:10364300121070E47BFF7A7FF9F890040A121023BA
:07365300120F43AE02AF03AA
:01365A00224D
:042122004107E90088
:103D1500E4F5849007E9F0F5BAF5BB75BCC075E824
:023D25008022FA
:031A30000230760B
:10307600C0E0C0F0C083C082C0D075D000C000C020
:1030860001C002C003C004C005C006C007758400A5
:1030960053E8DF9007E9E025E024D9F582E4340718
:1030A600F583E5BFF0A3E5BEF09007E9E004F0C3C1
:1030B60094084005E4F0121BDB9007E9E0F5BBD06D
:1030C60007D006D005D004D003D002D001D000D05E
:0A30D600D0D082D083D0F0D0E032D9
:0F1A2100E4F58475D48075840175D480F5842232
:103BEA007808E0FEA3E0A60608F62292AFAF028F9D
:063BFA00B1AF038F84222D
:10313F00AB84AAB1A2AF92169008781210709008C3
:10314F007A123BEA53B10F900879E0700543B11042
:10315F00801990087AE030E70543B130800D43B114
:10316F002090087AE04480F0123BEAE4F584C2AF85
:10317F0043B701758F037808E6FE08E6F5828E8364
:0C318F00E4F053B7FEF58FA216123BF5DA
:01319B002211
:10199100AB84AAB1A2AF92179008231210709008DD
:1019A10022E0F9FF3395E0FEEFF44E6053900825F5
:1019B100780A123BEC53B10F900824E0700543B153
:1019C100108020900825E030E70543B130801443B2
:1019D100B120900825E04480F0E0FEA3E0780AA65B
:1019E1000608F6E4F584C2AF43B701758F01780AA2
:1019F100E6FE08E6F5828E83E9F053B7FEE4F58F43
:051A0100A217123BF5E5
:011A060022BD
:103D7A000001FF00FF000001010000FF00FF010039
:10212600032500002B032800002B410832F8410844
:1021360030F8C10FC10E410837004108310042088E
:10214600350000C10D410833004108340001240068
:103B59009400E09408900832E022E52885298385BD
:093B69002A82229008830210C98F
:101BDB00900832E0900830F0A20F920E9007D9E0F7
:101BEB00FFA3E090083CCFF0A3EFF0E4FDFF121E43
:101BFB00DAC39007DDE094084004D20F8002C20FD5
:101C0B00A20FB00E50057F071232B0D39007E0E061
:101C1B009007DF123B5940054408F0800354F7F05E
:101C2B00D39007E2E09007E1123B5940054410F0D6
:101C3B00800354EFF0D39007E4E094009007E31295
:101C4B003B5B40054420F0800354DFF0D39007E664
:101C5B00E094009007E5123B5B40054440F08003A5
:101C6B0054BFF0D39007E8E094009007E7123B5B7A
:101C7B0040054480F08003547FF0900832E0FC5420
:101C8B00187004A37403F0900830E0FE6CFDEE5D59
:101C9B00900893F0AF05EC5FA3F030E31890083396
:101CAB00E070047F01800B900833E054FEF0700568
:101CBB007F0A1232B0900893E030E5057F031232B1
:101CCB00B0900893E030E6057F041232B090089391
:101CDB00E030E7057F051232B0900837E09008310D
:101CEB00F0A3E0F45410900837F0900833E0706ADA
:101CFB00900837E06033900831E07006900835F0BB
:101D0B00A3F0900835E475F001120E71D3900836EC
:101D1B00E09478900835E064809480403D200D3A43
:101D2B007F061232B0D20D8031900837E0702B90C5
:101D3B000831E06025900835E0FEA3E0FFD3940660
:101D4B00EE648094804011EF9478EE648094805020
:101D5B00077F021232B0D20DC20D900894E030E42E
:101D6B0010900833E0600A54FDF070057F0A1232C0
:011D7B00B0B7
:011D7C002244
:1032B000AB25E5272401F9E43526FA90088312119D
:1032C00000123B6C90004BEB7008E965827003EADA
:1032D0006583700BFB7A00792B9008831211001222
:1032E0003B6C123B636B7008E965827003EA65838F
:1032F0006013AB25AA26A927EF120DF8123B6C8BA1
:05330000258A26892743
:0133050022A5
:10349C0053E6F7AB25AA26A927123B636525700ACC
:1034AC00E52765827004E52665837003FF80287824
:1034BC0028E475F0011210B9120DB2FF90004BE523
:1034CC0028700AE52A65827004E52965837008F581
:0A34DC0028752900752A2B43E60825
:0134E60022C3
:1038750053E6F7123B636525700AE52765827004F8
:10388500E52665837003FF800AAB28AA29A92A12B9
:063895000DB2FF43E6083E
:01389B00220A
:0F3D8A00C39007E5E0940840037F00227F0122E9
:031A1E00022A3663
:102A3600C0E0C0F0C083C082C0D075D000C001C065
:102A460002C003C005C006C007C2AF30DF02C2DF46
:062A560020D90330D8680E
:102A5C00E5905403900886F0C2D8C2D9900834E0AF
:102A6C00FF900886E0FD6F5403604D53E6F7EF7559
:102A7C00F004A47E00540CFFED5403FDEF4D247ABA
:102A8C00F582EE343DF583E493FF900887F0A3E5DF
:102A9C0024F0EF2524F524E0652430E1109008871C
:102AAC00E0B401047F0880027F091232B0900886DE
:082ABC00E0900834F043E60845
:102AC400D2AFD007D006D005D003D002D001D0D0E9
:092AD400D082D083D0F0D0E032B2
:103C9300E475F001120E8785F082F58322EEF0A31E
:043CA300EFF0A32279
:0B3E2400AF01AE027C00E4FD02313F64
:053C2B009008A6EDF079
:103C3000AF01AE027C00E4FDE0900822F002199191
:10330600900864123CA0ECF0A3EDF0A3EAF0A3EB66
:10331600F0900868E07002A3E0603A900864E0FE6E
:10332600A3E0AA06F97B01A3E0FEA3E0F5828E8363
:10333600E0FD123C2B90086874FFF5F0120E7190B8
:103346000866E475F001120E71900864E475F001E8
:06335600120E7180BC2282
:081A0700E4900000F0A3F022BE
:1037AA00900000E0FEA3E0AA06F97BFF123E2490F7
:1037BA000000E0FEA3E0FF7C007D027B007A041299
:0A37CA003306E4900000F0A3F022A3
:0D2F8800900851EDF090084FEEF0A3EFF02F
:102F9500EE54FCFE900000E0FCA3E0FD7002EE6C38
:102FA5006044ED4C60031237AA90084FE0FEEE54E2
:102FB500FCFE7F00900000F0A3EFF0900852123C59
:102FC500A07400F0A37402F07FFF7E0390085212F4
:102FD5003C93E493FD900854123C93EDF0EF1F7081
:102FE500011EEF4E70E6900851E0FF90084FE0FC9F
:102FF500A3E0FDEC5403FC74022DF58274003CF54E
:0330050083EFF066
:0130080022A5
:10365B00900856123CA012110090085B74FFF5F015
:10366B00120E8745F06020900856E475F001120E9B
:10367B0087AFF0FE900858E475F0011210D2120DCE
:08368B00B2FD122F8880D2224B
:1030090012102F12352F9007CD1210709007C6E0BD
:1030190025E0243CF582E43408F583E0FEA3E022B0
:10302900FBC374FF9BFF740F9EFEE49400FDE494C0
:1030390000FC229007C6E025E02438F582E4340834
:10304900229007C5E025E0242AF582E4340722E42A
:103059007F01FEFDFC12102FC3020FD5E47BFF7A1E
:0D3069000FF9F8229007CD12102F020EB8BB
:081EDA009007C5EFF0A3EDF045
:101EE200123040123022FBAA06E4F9F8123015FF34
:101EF200E4FCFD120EAA9007C9121070E49007C705
:101F0200F0A3F07F0FFEFDFCA312305E40089007A5
:101F1200C7E4F0A304F074FF7FF1FEFDFC9007C953
:101F220012102FD3120FD5500874FF9007C7F0A3D9
:101F3200F09007C7E0FEA3E0FF4E700302202DEFF2
:071F4200F47002EEF470548C
:101F490012303C123022FFE4FCFD9007D5121070CC
:101F59009007D5123058500A9007D512107C00000E
:101F6900000112304A123022FFE4FCFD12306612E1
:101F79000EB89007D5123009FFE4FCFD12306D90C0
:101F890007D11210701230659007D1121023123543
:011F99002F18
:0F1F9A000220009007C7E07004A3E064017064A8
:101FA90012304A123022123029123065120EB890BE
:101FB90007CD12107012303C1230221230299007CE
:101FC900D11210709007D1123058500A9007D112CF
:101FD900107C000000019007CD1210239007D11248
:101FE900300912302912306D12306512352FC37441
:101FF900FF9FFF740F9EFE12304AF583EEF0A3EFA8
:04200900F0121A1B9C
:10200D009007C6E0FF25E0243CF582E43408F58313
:10201D00E0FCA3E0FDEF123040F583ECF0A3EDF012
:01202D002290
:103BA30000320078007D00830088009100A400B6F5
:083BB30000C800DB00EE00FF7A
:103C000033FE74A32FF582743B3EF583740193C495
:063C1000F8540FC8682201
:103BD300E4F5B0F5A0F590F584F5D3F5D27584013D
:073BE300F5D3F5D2F58422B1
:1017BF00E4900861F0FF90072CE0FCA3E0FBAA0483
:1017CF0090071DE0FEB401057402FF8008EEB4021D
:1017DF0004EF4401FF90071CE0FE7006EF4408FF82
:1017EF008008EEB40104EF4404FF900727E0146073
:1017FF001014601314601624037016EF4410FF804A
:10180F0010EF4420FF800AEF4440FF8004EF448034
:10181F00FF8FB0C3EB9448EA9400400890086174BE
:10182F003FF08058C3EB943CEA9400400890086165
:10183F00749FF08047C3EB9430EA940040089008FF
:10184F006174CFF08036C3EB9424EA940040089083
:10185F00086174E7F08025C3EB9418EA9400400800
:10186F0090086174F3F08014C3EB940CEA94009029
:10187F000861400574F9F0800374FCF07C007D0C66
:10188F00AF03AE02120E1CED25E0FFEC123C00FE82
:10189F00E493C454F048900862F0A3CEF0AE04AFC6
:1018AF0005C3740B9FFFE49EFEEF25E0FFEE123C95
:1018BF0000FFE493C454F048FEC3EB940CEA940089
:1018CF004008EB9418EA94004028C3EB9424EA9460
:1018DF00004008EB9430EA94004017C3EB943CEAC5
:1018EF0094004008EB9448EA94004006EB64544A95
:1018FF007013900862E0FDA3E090085DCDF0A3EDBA
:10190F00F0A3EE801390085DEEF0A3EFF090086265
:10191F00E0FFA3E090085FCFF0A3EFF075A0FFE426
:10192F00F58490085DE0FEA3E0FF8ED38FD275841F
:10193F0001A3E0FEA3E0FF8ED38FD2E4F584A3E0F2
:10194F00F5A030030543901080035390EF900426C9
:10195F00E014600C1460112402701353903F800E3A
:10196F005390BF439080800653907F439040300B3D
:10197F000543900480035390FB90041BE024FF92D7
:01198F0093C4
:011990002234
:0B2B8100900817EDF0900814121100EE
:102B8C00AF0190081CEAF0A3EFF090081874FF1244
:102B9C00103DEC4D4E4F60789008141210C9E9248A
:102BAC0028F9E43AFAC003C002C00190081CE0FE08
:102BBC00A3E0FFF9D082D083D0E064017008E9650E
:102BCC00827003EE658360209008141210C9E9240A
:102BDC0042F9E43AFAEB8A83898264017008EF6562
:102BEC00827003EE658370098F828E837404F0808B
:102BFC0012900817E0FF90081CE0FCA3E0F5828C13
:102C0C0083EFF090081CE475F001120E71022B9604
:012C1C002295
:0421560041084000FC
:1039B900900895EFF0A3EDF07F0A12319C900895DD
:1039C900E0FF12319C900896E0FF12319C023DC441
:103B2600900840E0701304F07F0212319C123DC4ED
:0A3B3600E4900840F0900457F022DC
:0636C700123E5FEF6027D8
:1036CD009008977408F0A37441F01237FD90089795
:1036DD00E475F001120E8785F082F583EFF0123E4E
:0736ED0065EF70E67F01228A
:0336F4007F002232
:103C40009008A7EFF07F2F12319C9008A7E0FF1299
:053C5000319C023DC49F
:103C55009008A8EFF07F3012319C9008A8E0FF1281
:053C6500319C023DC48A
:083E430018100C08060403022C
:06215A004108AA00C118B3
:103D4900F9F812352F90086F12107090086F021051
:013D59002346
:1036F700900001120DCBFF9008A9F0BFF803022636
:10370700689008A9E0B4FA03023CBA9008A9E0B4AB
:0F371700FC03023DDF9008A9E0B4FB03123DB6AE
:013726002280
:103CBA00D218E49008AAF090071CE0B40204A37496
:033CCA0001F022E4
:0D3DDF00C21890071CE0B40203E4A3F02218
:0E3DB600D21890071CE0B40204A37401F0229E
:102668002018030227369008AAE0FF04F0EFB460B0
:0F267800037401F090071CE06402600302273630
:1026870090072CA3E0FF75F00C120D90900873F0E3
:1026970090072AE0FEA3E0FFE42FFBEE34F8FAE40C
:1026A70034FFF9E434FFF89007DBE0FEA3E0FFE432
:1026B700FCFD120EB8123D4EE4FB7A08123D49E4C8
:1026C7007B2D7A02123D49900873E02FF0E0FFC39B
:1026D700648094805004E4F0800ED3EF6480948784
:1026E70040069008737407F0900873E0FF3395E095
:1026F700FE74432FF582743E3EF583E493FD3395D4
:10270700E0FC9008AAE024FFFFE434FFFE120E1C51
:10271700ED701C90071DE064016011900426E0FF36
:0F27270064016008EF640260033006031214E4DB
:012736002280
:1037270075840F758A83E4F589F58475B7307584D8
:103737000F438901758D01758E04758F017FFFDF3A
:0C374700FE438902E58930E4FB7597021F
:013753002253
:0821600041089A0041089900B2
:1023CF0090650175F05DED1210ADEC75F05DA42513
:1023DF0083AF82900806F0A3EFF09007FEE075F050
:1023EF005DA42401F9746535F0FA7BFF22E075F0E6
:1023FF005D9065011210ADAF82AE8322900717E496
:10240F0075F001020E717A07791C7B0190085BE46D
:10241F00F0A3229006B3E475F0011210D2AE02AF12
:10242F000122F074FAA3F0A3E4F0A322E024FFFF4B
:10243F00E434FFFE9007FFE0FCA3E0FD22900717B6
:10244F00E0FCA3E0FDC3945DEC940022E475F00181
:10245F00120E8785F082F583E4932224FFFEE43485
:10246F00FF9007FFF0A3CEF022900803121100E4B3
:10247F00900801F0A3F022AD04EDFFEEF0A3EFF012
:10248F0022E4900717F0A3F022AF05E4F0A3EFF0DA
:10249F00E07F00FE2274B82DF582E43406F5832226
:0A24AF009FEE6480F8EC6480982230
:102ADD0090089B7401F0E4A3F0121A077E657F0045
:102AED007A08799B12241904F012365B7E707F44AC
:102AFD007B017A08799C12241B04F012365B123785
:102B0D00AA7B017A07791C90081812107C0000002E
:102B1D005DE4FD122B81E490071EF0900727F090E5
:102B2D00071F12243174FAF0A3E412243174FAF061
:102B3D00E490071DF090071CF0900728F0A3F074A7
:102B4D0008122434F0A3742AF0E4FFEF25E0242EBC
:102B5D00F582E43407F583E4F0A3F074602FF58279
:102B6D00E43407F583E4F00FEFB419DF123E2F7F45
:042B7D001E0236936B
:103B7200907044E493600C906500E49364016003E8
:093B8200122ADDE490071AF0227A
:0536930090089DEFF01E
:10369800121A07E490089EF090089DE0FFA3E0FE50
:1036A800C39F501875F05DEE122400122415745D46
:0F36B800F012365B90089EE004F080DC0237AA27
:1039D90030021220101990041C740AF090045774D4
:1039E90001F0D210222001077FBB1234E7D2012255
:031A1B000239D9B4
:0E3D9900E4FFFE0FBF00010EBE01F8BFF4F5FF
:013DA70022F9
:103BBB00C21090071A1223EC781C7C077D017E0043
:083BCB007F5D120D6A022E79E4
:103C6A00121A0790071A1223FC122415745DF01217
:053C7A00365B0237AAD1
:0B3E2F00123C6AC210200202C20122F5
:082737009007FAEFF0A3EDF0AA
:10273F00A2AFE433900808F0C2AF9007FAE0FFD3DE
:10274F009B4033EF12246AEB149007FEF09007FBC7
:10275F0012243BD31224AF50581223CF12247812D5
:10276F0027C940FB1237AA9007FF12240E9007FECD
:10277F00E004F002275C9007FBE012246A9007FD4B
:10278F00E014A3F09007FA12243BC31224AF4021A8
:10279F001223CF1224781227C940FB1237AA9007B1
:1027AF00FF74FFF5F0120E719007FEE014F0022790
:0927BF0093900808E024FF92AF9A
:1027C80022900803E475F0011210D2AE02AF019016
:1027D8000806E475F001120E8785F082F583E4930C
:1027E800FD122F88900801E475F001120E71C39054
:0C27F8000802E0945D900801E0940022CB
:052804009006B2EDF0AA
:10280900A2AFE433900719F0C2AFEF14900715F0A7
:10281900EB14A3F09006B2E014FF900715E0D39FE4
:1028290040030228C3A31223FC12249012244C5003
:10283900190FEFAA0670010E14F5828A83E493FB3F
:102849001224A4EBF012240B80E29007161223EC59
:102859009006B31211009007151223FC9006B6EEEC
:10286900F0A3EFF01224901224229006B612245BF2
:10287900FD122F8812240BC3900718E0945D90076E
:1028890017E0940040E19007151223EC9006B3126B
:10289900110012249012244C50101224221224A444
:1028A900E0FD122F8812240B80EB1237AA9007152E
:1028B900E004F0A3E004F002281D900719E024FFCA
:0228C90092AFCC
:0128CB0022EA
:072D4E00900809EBF0AC074F
:102D5500A312249890080AF0A3EFF090080A122411
:102D650086A2AFE433900813F0C2AF900812740F37
:102D7500F0121A079008121223EC90080E12110097
:102D8500E490080CF0A3F090080AE0FCA3E0FFEC47
:102D9500FD900809E0FBE490087FF0D2121224B9F7
:102DA500900811EFF0FD90080E122425122F88903F
:102DB500080A12240E90080C12240EC390080DE088
:102DC500945D90080CE0940040BD1237AA9008125B
:0E2DD500E004F0E0C3941E4098123573D2AFB4
:012DE30022CD
:072CB700900827EBF0AC07C9
:102CBE00A2AFE43390082FF090082A1224989008BF
:102CCE002AF0A3EFF090082A122486C2AF90082EA5
:102CDE00740FF090082EE0FFC3941E505775F05DF0
:102CEE00EF12240090082CEEF0A3EFF0E4900828E9
:102CFE00F0A3F090082AE0FCA3E0FFECFD9008277B
:102D0E00E0FB90082C12245B90087FF0C212122474
:102D1E00B990082A12240E90082812240EC3900887
:102D2E0029E0945D900828E0940040C790082EE0BA
:0F2D3E0004F0809F12357390082FE024FF92AFAE
:012D4D002263
:0724B90090087CEFF0A9057B
:1024C000C21320C3FD20C5FAC2C4D2C5E4FFFD304B
:1024D000C3FD30C3FDE5C154F8FC64086004ECB4EE
:1024E0001013EFB40105EB44018003EB54FEF5C279
:1024F0007D01022587ECB4180B89C27D02C2C4C2DB
:10250000C5022587ECB420028045EC6428703CEDC0
:10251000B4020E90087CE0F5C27D03C2C5C2C4803F
:1025200066EDB4031B301208D2C57F01C2C48057C8
:1025300090087FE0F5C2C2C57D04E4FFC2C48047B5
:10254000ED64047042D2C47D05803CECB4300AD204
:10255000C4D2C57D08E4FF802EECB438028024ECA0
:10256000B44006C2C2C2C5801EECB448028014EC5E
:10257000B450028004ECB4580AD2C47D07AEC2C283
:10258000C28004D2C4D2C5C2C3ED64076008ED6442
:082590000560030224D2AF062E
:012598002220
:0A2168004107810041079A00C115EC
:10340100900784E475F001120E8785F082F583221E
:103411009007847407F0A3749BF02290077BE475F6
:10342100F001120E717E077FAF90077BE0229007BB
:103431007FE0FFA3E090077B2290077FE0FEA3E0FF
:0E344100FF90077B22E0F5C290077BE06E2231
:103A6C00AF84E4F584C2C343E60243F60275C30196
:0B3A7C0075C04475CF8F43C3018F84D9
:013A8700221C
:103573007E077F8690077DEEF0A3EFF0900782EE43
:10358300F0A3EFF0900779EEF0A3EFF07E077F9BB7
:1035930090077FEEF0A3EFF0900784EEF0A3EFF037
:0D35A30090077BEEF0A3EFF0C214023A6C2B
:10389C00900782123404EFF0900782123404EDF09A
:1038AC00900782E0B4070FA3E0B49A0A90078274E1
:0738BC0007F0A37486F0225F
:0D3DC400AF84E4F584C214C2C4D2C58F845C
:013DD10022CF
:10319C0020142FD21412340174FFF07C077DAF90F1
:1031AC000784E0B50408A3E0B5050312341112340A
:1031BC0001E4F0900784E0B50408A3E0B505031220
:1031CC003411123401E4F0900784E0B40708A3E052
:1031DC00B4AF03123411123401EFF0900784E0B451
:0D31EC000708A3E0B4AF031234117F0122E5
:1037540090077DE0FCA3E0FD900779E0B50408A3A1
:10376400E0B505037F002290077DE0FCA3E0F5822D
:0C3774008C83E0B507037F01227F002258
:1037FD0090077DE475F001120E7190077D1234046F
:10380D00E0FF90077DE0B4070FA3E0B49A0A90079C
:08381D007D7407F0A37486F02E
:013825002280
:063E5F007FFF1237542220
:063E6500E4FF12375422B5
:031A1800021A3679
:101A3600C0E0C0F0C083C082C0D075D000C000C076
:101A460004C005C006C00753E6F7E5C154F81211F5
:101A5600091B9C001A94081A94101ABD181AE4203F
:101A66001AEA281B47301B4C381B56501B56581B6E
:101A760062601B58681B62701B58781B56801B716E
:101A8600881B56901B71981B84A000001BC1C2C501
:101A960012341CB5060BA3E0B5070690077B12347B
:101AA6001490077B1234041234467003A3E06F606F
:101AB60003021BC1021B3E12341CB5060BA3E0B584
:101AC600070690077B12341490077B1234041234F5
:101AD600467003A3E06F6003021BC1021B3E123473
:101AE6002FCF801690078412343DE0FCA3E0FDB5AD
:101AF6000713ECB5060F90077FEEF0A3EFF0C2C513
:101B0600D2C4021BC18D828C83E0B4FF07C2C4D24B
:101B1600C5021BC112341CB5060BA3E0B50706901F
:101B2600077B12341490077B123404123446700378
:101B3600A3E06F6003021BC190077B123414021BE3
:101B4600C112342F802F12342FCFF0A3EFF0806B09
:101B5600801012342FCFF0A3EFF0D215ADC27FFF65
:101B66008004ADC2E4FF12389C8050900779E0FFF4
:101B7600A3E0900782CFF0A3EFF0D2C4803D900798
:101B860082E0FFA3E0900779CFF0A3EFF030152BAA
:101B9600D2C5C215802512343AEEF0A3EFF09007B5
:101BA60079E0FDA3E0900782CDF0A3EDF0D2C4A3C7
:101BB600E06E7003A3E06F6002D2C5C2C343E608BD
:101BC600D007D006D005D004D000D0D0D082D083A4
:051BD600D0F0D0E03268
:10390F0012343AE0FCA3E0FDB50719ECB5061590AB
:10391F000784E0FEA3E0FFEDB50709ECB50605202F
:06392F00C502D322C322F1
:100C1A0002112FE493A3F8E493A34003F68001F2B0
:100C2A0008DFF48029E493A3F85407240CC8C333DB
:100C3A00C4540F4420C8834004F456800146F6DFAA
:100C4A00E4800B010204081020408090202EE47EEC
:100C5A00019360BCA3FF543F30E509541FFEE4939F
:100C6A00A360010ECF54C025E060A840B8E493A366
:100C7A00FAE493A3F8E493A3C8C582C8CAC583CA91
:100C8A00F0A3C8C582C8CAC583CADFE9DEE780BE49
:01217200006C
:100C9A00E709F608DFFA8046E709F208DFFA803E3C
:100CAA0088828C83E709F0A3DFFA8032E309F60829
:100CBA00DFFA8078E309F208DFFA807088828C8391
:100CCA00E309F0A3DFFA806489828A83E0A3F60845
:100CDA00DFFA805889828A83E0A3F208DFFA804C1F
:100CEA0080D280FA80C680D4806980F280338010F6
:100CFA0080A680EA809A80A880DA80E280CA80335F
:100D0A0089828A83ECFAE493A3C8C582C8CCC583D6
:100D1A00CCF0A3C8C582C8CCC583CCDFE9DEE780A6
:100D2A000D89828A83E493A3F608DFF9ECFAA9F025
:100D3A00EDFB2289828A83ECFAE0A3C8C582C8CC7B
:100D4A00C583CCF0A3C8C582C8CCC583CCDFEADE94
:100D5A00E880DB89828A83E493A3F208DFF980CCF6
:100D6A0088F0EF60010E4E60C388F0ED2402B404EF
:100D7A000050B9F582EB2402B4040050AF23234596
:060D8A008223900CEA73C5
:100D9000C2D530F707B2D563F0FF05F030E70CB2EB
:100DA000D5F4048463F0FF05F080018430D502F4AB
:020DB00004221B
:100DB200BB010689828A83E0225002E722BBFE023F
:090DC200E32289828A83E4932272
:100DCB00BB010CE58229F582E5833AF583E02250DD
:100DDB0006E92582F8E622BBFE06E92582F8E22227
:0D0DEB00E58229F582E5833AF583E4932241
:100DF800BB010689828A83F0225002F722BBFE01DA
:020E0800F322D3
:100E0A00EF8DF0A4A8F0CF8CF0A428CE8DF0A42EFC
:020E1A00FE22B6
:100E1C00BC000BBE0029EF8DF084FFADF022E4CCBA
:100E2C00F875F008EF2FFFEE33FEEC33FCEE9DEC83
:100E3C00984005FCEE9DFE0FD5F0E9E4CEFD22EDC9
:100E4C00F8F5F0EE8420D21CFEADF075F008EF2F13
:100E5C00FFED33FD4007985006D5F0F222C398FD04
:050E6C000FD5F0EA22A1
:100E7100C5F0F8A3E028F0C5F0F8E582158270020C
:060E81001583E038F022A9
:100E8700A3F8E0C5F025F0F0E5821582700215831E
:060E9700E0C838F0E8227B
:0D0E9D00EF2BFFEE3AFEED39FDEC38FC22A4
:0E0EAA00C3EF9BFFEE9AFEED99FDEC98FC2243
:100EB800E88FF0A4CC8BF0A42CFCE98EF0A42CFCD9
:100EC8008AF0EDA42CFCEA8EF0A4CDA8F08BF0A457
:100ED8002DCC3825F0FDE98FF0A42CCD35F0FCEBB6
:100EE8008EF0A4FEA9F0EB8FF0A4CFC5F02ECD397B
:0F0EF800FEE43CFCEAA42DCE35F0FDE43CFC22E8
:100F070075F008758200EF2FFFEE33FECD33CDCCA1
:100F170033CCC58233C5829BED9AEC99E582984024
:100F27000CF582EE9BFEED9AFDEC99FC0FD5F0D601
:100F3700E4CEFBE4CDFAE4CCF9A88222B800C1B92B
:100F47000059BA002DEC8BF084CFCECDFCE5F0CB69
:100F5700F97818EF2FFFEE33FEED33FDEC33FCEBA2
:100F670033FB10D703994004EB99FB0FD8E5E4F95D
:100F7700FA227818EF2FFFEE33FEED33FDEC33FC4A
:100F8700C933C910D7059BE99A4007EC9BFCE99A3E
:100F9700F90FD8E0E4C9FAE4CCFB2275F010EF2F83
:100FA700FFEE33FEED33FDCC33CCC833C810D70783
:100FB7009BEC9AE899400AED9BFDEC9AFCE899F8BE
:0E0FC7000FD5F0DAE4CDFBE4CCFAE4C8F92251
:10352F00C2D5E830E70FB2D5E4C39BFBE49AFAE4C7
:10353F0099F9E498F8EC30E717B2D5123565120F08
:10354F0043E4C39BFBE49AFAE499F9E498F8800307
:10355F00120F4330D50DE4C39FFFE49EFEE49DFDA3
:04356F00E49CFC22BA
:100FD500EB9FF5F0EA9E42F0E99D42F0EC6480C893
:060FE50064809845F02233
:100FEB00EB9FF5F0EA9E42F0E99D42F0E89C45F05C
:010FFB0022D3
:100FFC00E8600FECC313FCED13FDEE13FEEF13FFD3
:03100C00D8F122F6
:10100F00E86010ECA2E713FCED13FDEE13FEEF13F7
:04101F00FFD8F022E4
:0C102300E0FCA3E0FDA3E0FEA3E0FF2240
:0C102F00E0F8A3E0F9A3E0FAA3E0FB2244
:10103B007401FF3395E0FEFDFCA3A3A3E0CF2FF0DB
:10104B00E582158270021583E0CE3EF0E5821582B3
:10105B0070021583E0CD3DF0E58215827002158399
:05106B00E0CC3CF02286
:0C107000ECF0A3EDF0A3EEF0A3EFF022F3
:10107C00A8828583F0D083D0821210931210931221
:10108C001093121093E473E493A3C583C5F0C58346
:10109C00C8C582C8F0A3C583C5F0C583C8C582C8BE
:0110AC002221
:0C10AD00A42582F582E5F03583F583224E
:1010B900FAE6FB0808E6F925F0F618E6CA3AF62238
:0910C900E0FBA3E0FAA3E0F92228
:1010D200F8E0FBA3A3E0F925F0F0E58215827002A7
:0710E2001583E0FA38F0224B
:1010E900F8E0FBA3A3E025F0F9F0E5821582700290
:0710F9001583E038FAF02234
:09110000EBF0A3EAF0A3E9F022F0
:10110900D083D082F8E4937012740193700DA3A375
:1011190093F8740193F5828883E473740293686089
:06112900EFA3A3A380DF89
:00000001FF
